:020000040000FA
:060000000219FD020310CD
:030013000204FFE5
:03001B0002008D53
:03002B000202D5F9
:03005B0002050E8D
:030073000202FD89
:100080000406080C10182030406080A0C0C2AFC227
:10009000A853E6EFC28E856B8BC0D0D2D3C0E0C030
:1000A000F0C2CAA8CCA9CDD2CAD2AF758A00C3E823
:1000B000956CF8E9956DF9C3E913F9E813F8E5666D
:1000C0006007C3E913F9E813F8E97025E8956E4075
:1000D00020956E501CE582B410177C007B007A00DE
:1000E0007908900000A86AE5667004C3E813F80177
:1000F000FA900000D2A8D2AA61BAE0FDC39CC398CE
:1001000040EF98EB33FB0582E0FCC39DC39840E1D0
:1001100098EB33FB0582E0FDC39CC39840D398EB7A
:1001200033FB0582E0FCC39DC39840C598EB33FBCD
:100130000582E0FDC39CC39840B798EB33FB058272
:10014000E0FCC39DC39840A998EB33FB0582E0FD1A
:10015000C39CC398409B98EB33FB0582E0FCC39D96
:10016000C398408D98EB33FB05822175900000D237
:10017000A8D2AA61BAE0FDC39CC39840EF98EA33C5
:10018000FA0582E0FCC39DC39840E198EA33FA0582
:1001900082E0FDC39CC39840D398EA33FA0582E01D
:1001A000FCC39DC39840C598EA33FA0582E0FDC3BD
:1001B0009CC39840B798EA33FA0582E0FCC39DC31C
:1001C0009840A998EA33FA0582E0FDC39CC39840A1
:1001D0009B98EA33FA0582E0FCC39DC398408D9852
:1001E000EA33FA0582EBC46B6A54F0F9EAC454F0BE
:1001F000C3996009900000D2A8D2AA61BAEBF4C4F6
:1002000054F0F9EAF4C4540F49FAEBF4C4540FFB68
:10021000C3EAF99460FAEB9400FB5020C3E97B0039
:100220007A0079006016C3135006F9C39552600A2C
:10023000E9F552755300790080020553303A27C31F
:10024000EA94D0F8EB9407F9400BE8FAE9FB203583
:1002500009D235415A303502C235203902B235C390
:10026000EA33FAEB33FBEB2B3B3BF9C3EB13FBEA33
:1002700013FAEA29FAEB3400FB30E3047AFF7BFF40
:10028000E5255403601B202A18E55D33F9EB700760
:10029000C3E99A4002E9FAE53CC4332AFAEB340098
:1002A000FBC3EA33C4540FF8EB33C454F048F8707E
:1002B00005EA60027801C3EB13FBEA13FA90000031
:1002C000D2A8D2AAE52260021522819E900000D217
:1002D000A8D2AA61BAC0D0C0E0C2CF0541E5236070
:1002E000021523C3E554600575550041F8E5552412
:1002F00001F55550037555FFD0E0D0D032C2AF5351
:10030000E67F7592FA7593FFC22053917FD2AF3288
:10031000C0E0E58A303408856B8BF0A3D0E032D0A2
:10032000E0C2AF53E6EFC0D0C0E0C0F0D2D3D2AF4E
:100330005388EFA88AA98C758A00758C00438810B1
:1003400030331FE8C4540FFAE9C454F04AFAC31317
:100350002AFAC3E833F8E933F9E82AFAE93403FB67
:1003600061AB30320FC3E833E933FAE82AFAE934F3
:1003700000FB61AB303115E875F056A4AAF0E975C1
:10038000F056A42AFAC5F03400FB61ABE875F02BF7
:10039000A4AAF0E975F02BA42AFAC5F03400C3131F
:1003A000FBEA13FAC3EB13FBEA13FAC3EB9409500D
:1003B00009C3EA949AEB940350160522E5227002D1
:1003C0001522C3E5229432500281F275540081F562
:1003D000E522600215223036067C007D0461EAAC1D
:1003E00031AD32303A04AC33AD34C3EA9CFAEB9D04
:1003F000FB9208AE60AF61303A425007203509D217
:10040000358108303502C235303504AE62AF632025
:100410003902B235C3EA33FAEB33FBA208500AEAD9
:10042000F42401FAEBF43400FBC3EA9428FAEB94C9
:1004300000FB501478007A007B008148A208500825
:1004400078007A007B00819EE52554036019202AFC
:1004500016E55DF9EB7007C3E99A4002E9FAE53C5D
:10046000C42AFAEB3400FBEA8EF0A4F9AAF0EB8E72
:10047000F0A42AFAC5F03400FBC3EB13FDEA13F82D
:100480000FEF146004C3E833F8C3E933EA33FAEB3F
:1004900033FBDFEDEB30E20678FF7AFF7B03885415
:1004A000D230E86003755500C3E55BFC955C400203
:1004B000AC5CC3EC95545008EC75F004A4FAABF0B6
:1004C000EAF4F8EBF45403F9C3E89414FAE994005D
:1004D000FB50047A007B00885689578A588B5975DF
:1004E000230AD0F0D0E0D0D053F7DF43F74043E603
:1004F000103275230AD0F0D0E0D0D043E61032C2DB
:10050000AAD28EC2CA85CC6C85CD6DD2CA32C2AF9A
:10051000C0D0C0E0D2D3A8F9E55A30E10AE5FA200C
:10052000E13520E032A12FE5FA30E12B20E028C3AD
:10053000E55713F8E55613F5FB88FCC3E55913F8A6
:10054000E55813F5E988EA85575A53F7BFD2A83022
:100550003402D2AA53E6EF53F7DFD0E0D0D0D2AFC7
:10056000327901801479038010790A800C791E8019
:10057000087964800479C880007817E4D5E0FDD854
:10058000FAD9F62278FF20282879A1E76023E548E8
:10059000601F74FF8548F084853FF030290375F0B3
:1005A00005A4F8C5F0600278FFC3E8955D5002A885
:1005B0005D885C22C3E54794E4E5489400E55C501F
:1005C0000314A1C5046002F55C2275E89022055E63
:1005D000C3E55E9408405330EDF4A8BDA9BE755E36
:1005E00000E9FA79A0E76041EA7006E55F601880EB
:1005F0000CC3E8955F600EE55F5005600A14800744
:100600000460FA8002E55FF55FC39569401B755B86
:10061000C0C394044013755B80C39404400B755BA6
:1006200040C394044003755B0022E55B2410500234
:1006300074FFF55B22743279A687F0A4C5F0A2F7A7
:1006400033F55D227547007548F022C2AFC2CAA8D3
:10065000CCA9CDAA4130CF010AD2CAD2AFAB42ACAD
:100660004388428943C3E89BF8E99C202808F93075
:100670002C02E15BC1B4AD448A44F9EA9DFA6006FC
:1006800078FF79FFC199AE45AF468B458C46A842AD
:10069000A943C3E89EF8E99FF9C3E54813FBE54782
:1006A00013FAE82AF547E93BF54850067547FF7508
:1006B00048FFE101AA47AB48AC47AD487E047F0242
:1006C000C3EB9404400D1E1FC3EB94084005202982
:1006D000021E1FC3ED13FDEC13FCDEF7C3EA9CFA08
:1006E000EB9DFBEF6009C3E913F9E813F8DFF7EAC4
:1006F00028FAEB39FB8A478B4850067BFF8B478BE8
:1007000048C3EB94025002D22C3028047F03E12C22
:100710007892E6FFC3E53D948240110FC3E53D9416
:10072000A040010FC3EF940640027F057E02E5481A
:10073000C4540FF9E548C454F0F8E547C4540F28F1
:10074000F8C3E89EFAE99400FB4009C3EA9401EB80
:10075000940050047A01E4FB0207A7AA47AB48EBD8
:10076000C4FEEAC4540F4EFCC3EA9CFAEB9400FBAF
:10077000C3E813C313F8EA28FAEB3400FB8A478B6B
:1007800048C3EB94024002C22C7802EBC4FE7B000B
:10079000EAC4540F4EFAC3EA98FA4005C3940150D4
:1007A000027A017892E6FF302002E1A7854E928519
:1007B0004F93D22043E680C3E49AF8E49BF9302CAF
:1007C00003020835E8FAE9FBD3E913FDE813FC88D6
:1007D0004E894FC3EF94036038EF20E00CE82CF80B
:1007E000E93DF9ECFAEDFB8013E828F8E939F9C3A3
:1007F000E82401F8E93400F97AFF7BFFC3EF9403A2
:10080000400F8A508B51884A894B8C4C8D4D020881
:100810006A885089518A4A8B4B8C4C8D4D302812F6
:100820007550F07551FF754CF0754DFF754EF075B4
:100830004FFF02086AE8FAD3E813FC884EC3EF942E
:10084000036021EF20E007E82CF8ECFA0155E828D6
:100850002401F87AFFC3EF940340098A50884A8C38
:100860004C02086A88508A4A8C4C302002016A7512
:100870003A02D22043E680E52554036034A847A914
:1008800048C3E913F9E813F8C3E913F9E813F8309A
:100890002804E92440F9C2AF53E67F759100C3E410
:1008A00098F594E499F595759104D22043E680D2A9
:1008B000AF22D221754900752000302B03752040EE
:1008C00001D0D221754900752040302B03752000DE
:1008D00078017901202C20E52554036002C221799A
:1008E00014E548C313700104F8C39414400278144B
:1008F000302804781B791B202010E549600C302833
:1009000003D53A04D222217711720549E59B544060
:10091000B52002216130280908C3E8994001180177
:10092000F720210A08C3E899400201D001F7C2214B
:1009300053E67F759100302C117594007595F8750C
:100940009104D22043E6800208D0E5487EFFC333FD
:100950004005C3334001FEC3E49E759400F5952124
:100960003FC3E5399401500201D030210201D0D8B3
:1009700002217501F7C222C2AF53E67F759100854F
:100980005094855195759104854A92854B93D22058
:1009900043E680D2AFE525540360072029020539DC
:1009A000801030220D202B0A20210715811581028D
:1009B000136E2278003021027801E53D75F007A41E
:1009C000F9E5F028F5F0E9A2F013A2F113A2F21371
:1009D000F53DC394785003753D78C3E53D953E40A1
:1009E0000CC286C290C29275D4FF75D50F3020021A
:1009F00021ED854C92854D93D22043E6802220380C
:100A000013C2AFC291D28775D4FF75D503D2AF752B
:100A10009F4241F2C2AFC291D29375D43F75D50FB8
:100A2000D2AF759F4241F2203813C2AFC29275D443
:100A3000FF75D50CD287D2AF759F5241F2C2AFC2BB
:100A40008675D4FF75D50CD293D2AF759F3241F223
:100A5000203813C2AFC287D29375D4FF75D50CD29C
:100A6000AF759F3241F2C2AFC293D28775D4FF7582
:100A7000D50CD2AF759F528079203813C2AFC29087
:100A800075D43F75D50FD293D2AF759F428063C2A4
:100A9000AFC29075D4FF75D503D287D2AF759F4290
:100AA0008050203813C2AFC293D29175D43F75D510
:100AB0000FD2AF759F52803AC2AFC287D29175D420
:100AC000FF75D503D2AF759F328027203813C2AF90
:100AD000C28675D4FF75D503D291D2AF759F32808F
:100AE00011C2AFC29275D43F75D50FD291D2AF75F6
:100AF0009F52227A147B7880127A107B8C800C7A39
:100B00000D7BB480067A0B7BC88000E564D5E001DC
:100B1000227902E4C291D5E0FDD290D5E0FDC290E9
:100B2000D5E0FDD291D5E0FDE920E002D28630E0AB
:100B300002D292E564D5E0FDE920E002C28630E011
:100B400002C2927496D5E0FDD9C9EAF8D5E0FDD885
:100B5000FBDBB8C29122C286C290C292C287C29108
:100B6000C29375D4FF75D50F22788076FF0876FF83
:100B70000876FF0876FF0876FF0876FF08760908F2
:100B800076FF087601788C76010876FF0876FF08F4
:100B900076FF0876FF0876FF0876030876FF08766A
:100BA000FF0876FF0876250876D008762808765064
:100BB0000876040876FF0876020876FF08767A0839
:100BC00076FF0876070876010876FF0876FF087634
:100BD0000008760022FA75F00CA4ABF0EAC333F8F3
:100BE000740133F9E8C333F8E933F9E8C32BF8E9C2
:100BF0003400F9227888E6C39403D23A5002C23A0C
:100C0000C238E630E102D238A23892397886E6144A
:100C10009000809378A6F67886E6F53FC39402505C
:100C200003753F02789CE6753EFFB40203753EA053
:100C3000B40303753E8278A0E6F8600674282409A0
:100C4000D8FCF5697896E671D588318932789EE6C8
:100C500071D5883389347897E671D58835893671AE
:100C600056223036117A007B007CFF7D007E009199
:100C7000C88B618A6022303A227896E6FA7B007847
:100C80009EE6FC7D00C3EA33FAEB33FBC3EC33FC96
:100C9000ED33FD7E0A91C88B638A627896303A0202
:100CA000789EE6FA7B007897E6FC7D007E00303A7D
:100CB00010C3EA33FAEB33FBC3EC33FCED33FD7EB8
:100CC0000A91C88B618A6022C3EC9EFCED9400FD02
:100CD000C3EC9AFCED9BFDC3EC9423ED940050040F
:100CE0007C237D00C3EC94FFED940140047CFF7DE8
:100CF000017BFF0B7A000AEA7009C3EC33FCED3389
:100D0000FD81F3EC8AF0A4AEF0ED8AF0A42E947C81
:100D100040E4EAF460DD22D236916212056D1205DC
:100D20006D7A007B007C10120565E5542AFA740088
:100D30003BFBDCF37C04C3EB13FBEA13FADCF7FFA9
:100D4000EB60027FFFC23691622278A5E6F9540378
:100D50007000E9540C7000E954307000E954C07020
:100D600000227567007568007597DE7597AD75810F
:100D7000C043FF8075EF0675A900715675803F75F9
:100D8000F1C375A4C075803F75D4FF75900075F2EE
:100D90000F75A50F75900075D50F75A60175E34009
:100DA00075E2027156E4F8F6D8FD71691213A37862
:100DB000988664753001C2AF12057551F312056D46
:100DC00051F912056D51FF12056DB14AC2AF756739
:100DD0000075680078FA79FA308007D9FBD8F702F5
:100DE0001C0071F4916278988664715675E4007500
:100DF0008811758E0475890975C80475910475D8B4
:100E00004075D90875F781759E0375960275DA42AB
:100E100075DB4275A82175E69075B801759B8075E4
:100E20009D0075D10C75BC5975BB1075E88075B205
:100E300001120561D2AF753C00C230120575C23196
:100E4000C232C233C234755200752200120571C31A
:100E5000E522940A5002E120D23175220012057178
:100E6000C3E522940A5002E120C231D23275220039
:100E7000120571C3E522940A5002E12075E48075E1
:100E80008851758E017589AA758C00758D00C2A96F
:100E9000D2ABD2AA756BC0756A14756E50C232D2CD
:100EA0003475220A120571756A10C3E522940A7519
:100EB00052007553004069758E0C756B80756A28F9
:100EC000756E2875220A120571756A20C3E5229491
:100ED0000A7552007553004047758E0C756BC075CE
:100EE0006A14756E1475220A120571756A10C3E5CD
:100EF00022940A755200755300402575E4007588E8
:100F000011758E04758909D2A9C2ABC2AAC234D2A6
:100F100033752200120571C3E522940A4002A1CC68
:100F2000120565203003020DCCC2AF51F351F351CD
:100F3000F3D2AF120575203403303A03020FDE12EC
:100F40000565788CE6C394015002E1DEE530C39478
:100F5000015002E1DE7567A57568F17F02D2369116
:100F600062120571C2AFC2369162C3E554947FD25A
:100F7000AF406B120561C2AF7105D2AFDFDFB117B1
:100F8000C3EF7897F61205751214907F0AD2369146
:100F900062120571C2AFC2369162C3E554947FD22A
:100FA000AF50E8120561C2AF51F312056951F3D297
:100FB000AFDFDAB117EF24037896F6F87997E7C335
:100FC00094234003985006E824237897F612057579
:100FD0001213EA1214BF1205719162020DCC7567EB
:100FE00000756800120571C3E55494014002E136B2
:100FF000C2AF710571057105D2AF1205757530006C
:10100000E4F537F5380537E537F4703F0538789A59
:10101000E67819146012783214600D787D14600837
:1010200078FA146003753800C3E53898401D120B38
:1010300056120561153875370078998664C2AF126B
:101040000B05D2AF78988664120571120569E52305
:101050007003020DCCC3E55294015014C3E55494BF
:101060000140A2120571E5237003020DCC02120E9D
:10107000C3E55294017017C2AF120B56789986647B
:10108000120AF378988664D2AF1205714100C3E565
:101090005294027017C2AF120B5678998664120AE6
:1010A000F978988664D2AF1205714100C3E5529475
:1010B000037017C2AF120B5678998664120AFF7834
:1010C000988664D2AF1205714100C3E55294047052
:1010D00013C2AF120B5678998664120B05D2AF1269
:1010E00005714100C3E55294057017C2AF120B564B
:1010F00078998664120B0578988664D2AF120571D0
:101100004100C3E55294077019C3E5539409500296
:1011100001557401303A0274037888F6C238C23936
:101120004100C3E55294087019C3E5539409500275
:1011300001557402303A0274047888F6D238D239F4
:101140004100C3E55294097017C3E5539409500256
:101150000155303A0BC37888E69402F6C23A410052
:10116000C3E552940A7016C3E55394095002015521
:10117000203A0A7888E62402F6D23A4100C3E552C2
:1011800094147025C3E553940950020155C2AF90E1
:101190001A0B740093D2AF7888F613C238C2394064
:1011A00002D2384002D2398057C3E55294157038C4
:1011B000C3E5539409404FC2AF901A0B740093D209
:1011C000AFF8B801027402B802027401B8030274E5
:1011D00004B8040274037888F613C238C239400296
:1011E000D2384002D2398018C3E552940C70117580
:1011F00067A57568F1C3E5539409400A71EAD2AF57
:101200007552007553007567007568000155C2AFCF
:10121000120B56E4D2AFE4F55EF524F525F53D75E5
:101220005E081205611205CA30EDFDA8BDA9BEE930
:101230007001F8885F1205CE755E08C2AF120635E0
:10124000855D5B855D5CD2AF303A07C238303502D0
:10125000D238D228753900120AA2120ACB120644DB
:1012600012064B12064412064B1206441208C21212
:1012700009B31209FE12064B1208B2202C03120504
:1012800084302C031205B41209B3120A2712064B3C
:101290001208C21209B3120A5012064B1208B212F7
:1012A00009B3120A7912064B1208C21209B3120AC4
:1012B000A212064B1205CA1208B21209B3120ACBC7
:1012C0001205CE12064B302827855D5B79187A0C03
:1012D000C3E53999400EC228D2298A3B855D5B85DA
:1012E0005D5C800CC3E5549401400302126C61768E
:1012F00030291F202B1CE53B147006C229D22A413D
:101300006CF53B203A07C3E5549401400302126C8C
:101310008064753C00203A0F78FA79A4E76002787F
:1013200003C3E55598504FE523604B303A172038FA
:1013300005203507800F303502800A202B07D22B7D
:10134000855D5B419C78F0302B05855D5B7820C323
:10135000E54898500302126C302B1BC22BC2383068
:101360003502D238D229753B12855D5B416C053C54
:10137000E55460026179753C00C2AF120B567524CA
:1013800000752500D2AF120571120B5678A4E660E5
:1013900006D287D291D293C3E53C94044003020D58
:1013A000CC0100901A0D78209123E520B4550AA3B2
:1013B0009123E520B4AA0280137567A57568F11220
:1013C0000B6971EA756700756800801D901A0378D3
:1013D000807B0A9123A308DBFA901A0F788C7B1A82
:1013E0009123A308DBFA901A2922C2AF9166914398
:1013F000901A0074109128A3743E9128A37421912F
:1014000028901A0378807B0A9127A308DBFA901AA8
:101410000F788C7B1A9127A308DBFA91799157906A
:101420001A2922E493F622E6438F01538FFDFFC36E
:10143000E583941C400122EF8567B78568B7F053B8
:101440008FFE22438F02438F018567B78568B7906F
:101450001A0DF0538FFC22901A0D74559128901A92
:101460000E74AA9128227A3079D07820901A40916F
:1014700023E520F709A3DAF7227A3079D0901A40D1
:10148000E7912809A3DAF9227C05120575DCFB2215
:10149000C2AF120AF3120AF9120AFF120B05120563
:1014A00069120AF3120AF9120AFF120B05120569F2
:1014B000120AF3120AF9120AFF120B05D2AF22C266
:1014C000AF120B05120AFF120AF9120AF31205698C
:1014D000120B05120AFF120AF9120AF31205691219
:0E14E0000B05120AFF120AF9120AF3D2AF220C
:1019FD00020D62103E21FFFFFFFFFFFF09FF01FFF8
:101A0D0055AA01FFFFFFFFFF03FFFFFF25D0285061
:0D1A1D0004FF02FF7AFF0701FFFF0000FF3A
:101A400023435F4C5F3230232020202020202020A1
:101A500023424C48454C492445464D3842313023B9
:101A60002020202020202020202020202020202076
:101C0000C2AFC2D37597DE7597AD7581C075A90057
:101C100043FF80752438752503B1DB7529A5752A26
:101C2000F143F10153A4FED28075D4FF75E3407DEA
:101C3000FA780379E67C10752200752300901DE880
:101C40007B06752498752501308002814820800824
:101C5000D8FBD9F9DCF781BA308008D8FBD9F9DC98
:101C6000F781BAB19BE493A3C39A6004DDC381BA40
:101C7000DBDBB18D600281317B08E493FAA3B16EA6
:101C8000DBF87A30B16E752200752300B18DEAFC65
:101C9000EBFDC3ED94FE400EB18D8A278B28ED300D
:101CA000E0048A828B83B18D7AC270D8C3ED94FE32
:101CB000601950CEBD0029EC600F7520007521FF22
:101CC000752900752A000200008100A827A92808AC
:101CD00009D804D90281DDB191EAF281D10D81A642
:101CE000C3ED94035051EDA2E092007AC5C3E582A2
:101CF0009400E583941C508C200010438F02438F86
:101D0000018529B7852AB7F0300027A827A9280818
:101D100009438F01538FFDD804D902A132C3E58353
:101D2000941C4003A3A117E28529B7852AB7F0A325
:101D3000A117538FFC81827AC1BD030CE493A3FAEF
:101D4000B152DCF8B14A81828184AA22AB23B16E00
:101D5000EBFAEA6222752608C3E52313F523E52290
:101D600013F52250066323A0632201D526EAB1DBD6
:101D7000B1DB75260AEAF4200102D280300102C2EA
:101D800080B1DBC3134002C201D526EB22B191EA38
:101D9000FB208002A191308002A196752608AE2416
:101DA000AF25C3EF13FFEE13FEB1DFB1DBC3EA13C0
:101DB0003080024480FA30E703632201C3E5231335
:101DC000F523E52213F52250066323A0632201D5F3
:101DD00026D9E52265236523F52222AE24AF250E00
:101DE0000FDEFEDFFCD20122424C48656C693437BD
:061DF0003164E8B10601B8
:00000001FF
